:100000000C942A000C9447000C9447000C94470071
:100010000C9447000C9447000C9447000C94470044
:100020000C9417020C9447000C9447000C94470062
:100030000C9447000C94B2010C9447000C944700B8
:100040000C9447000C9447000C9447000C94470014
:100050000C94470011241FBECFE5D8E0DEBFCDBF12
:1000600012E0A0E6B0E0ECE7F7E302C005900D92E5
:10007000AA32B107D9F714E0AAE2B2E001C01D929A
:10008000AB37B107E1F70E94E20F0C94BD1B0C9453
:100090000000CF93DF93CDB7DEB7EBE3F0E0108243
:1000A000EAE3F0E01082E8E3F0E01082E7E3F0E05A
:1000B0001082E5E3F0E01082E4E3F0E080EC80837E
:1000C000E2E3F0E01082E1E3F0E082E98083EFE434
:1000D000F0E080E18083EEE4F0E081E08083EDE415
:1000E000F0E01082ECE4F0E01082E7E4F0E010824F
:1000F000E6E4F0E01082EBE4F0E01082EAE4F0E005
:100100001082E9E4F0E087E08083E8E4F0E08AE24E
:100110008083EBE5F0E01082E5E5F0E01082E4E5B5
:10012000F0E01082EAE5F0E080E88083EBE2F0E0C6
:100130001082EAE2F0E088E98083E0E4F0E086E81B
:100140008083E0E4F0E01082E9E2F0E083E0808385
:10015000E9E5F0E088E08083E8E2F0E080E8808391
:10016000E0E5F0E01082A8E3B0E0E8E3F0E08081B1
:100170008B7F8C93A7E3B0E0E7E3F0E080818460BD
:100180008C93ABE3B0E0EBE3F0E080818F758C9370
:10019000AAE3B0E0EAE3F0E08081806A8C9378948F
:1001A000DF91CF910895CF93DF93CDB7DEB721973D
:1001B0000FB6F894DEBF0FBECDBF8983EBE2F0E04F
:1001C00080819927807290700097C1F3ECE2F0E093
:1001D0008981808321960FB6F894DEBF0FBECDBF14
:1001E000DF91CF910895CF93DF93CDB7DEB72297FC
:1001F0000FB6F894DEBF0FBECDBF9A8389830AC0C5
:10020000E981FA8180810E94D30089819A810196D7
:100210009A838983E981FA818081882389F78DE037
:100220000E94D30022960FB6F894DEBF0FBECDBF5A
:10023000DF91CF910895CF93DF93CDB7DEB72297AB
:100240000FB6F894DEBF0FBECDBF9A8389830AC074
:10025000E981FA8180810E94D30089819A81019687
:100260009A838983E981FA818081882389F78AE1E9
:100270000E94D30022960FB6F894DEBF0FBECDBF0A
:10028000DF91CF910895CF93DF93CDB7DEB7279756
:100290000FB6F894DEBF0FBECDBF6A837B838C831D
:1002A0009D830BC08A819B81AC81BD810197A1098F
:1002B000B1098A839B83AC83BD8380915204909162
:1002C0005304009741F48A819B81AC81BD810097E2
:1002D000A105B10539F78A819B81AC81BD81009769
:1002E000A105B10539F481E090E090933402809348
:1002F00033022DC080915F0490916004FC01E05BAB
:10030000FC4F8081898380915F0490916004019605
:100310009093600480935F0480915F0490916004E7
:1003200021E08030920721F41092600410925F0463
:10033000F894809152049091530401979093530440
:10034000809352047894898199279F838E838E812C
:100350009F8127960FB6F894DEBF0FBECDBFDF9109
:10036000CF9108951F920F920FB60F9211242F93E1
:100370008F939F93EF93FF93CF93DF93CDB7DEB728
:100380002297DEBFCDBFEBE2F0E080818A83ECE212
:10039000F0E0808189838A8199278C719070009721
:1003A000B1F580919A0290919B02FC01E05BFC4FB9
:1003B0008981808380919A0290919B02019690930B
:1003C0009B0280939A0280919A0290919B0221E075
:1003D0008030920721F410929B0210929A02809131
:1003E00052049091530401969093530480935204C5
:1003F000809152049091530421E08030920739F4A7
:10040000109253041092520481E080934E0322967E
:10041000F894DEBFCDBFDF91CF91FF91EF919F9117
:100420008F912F910F900FBE0F901F9018951F92D4
:100430000F920FB60F9211242F938F939F93EF93E8
:10044000FF93CF93DF93CDB7DEB7809137029091C2
:10045000380201969093380280933702ECE4F0E082
:10046000118210828091390290913A02009741F4F2
:1004700080913702909138022FE0803A920719F468
:10048000EFE4F0E01082DF91CF91FF91EF919F9127
:100490008F912F910F900FBE0F901F901895CF93B3
:1004A000DF93CDB7DEB725970FB6F894DEBF0FBE4A
:1004B000CDBF19821A8223C089819927FC01E45C8F
:1004C000FD4F8081282F33278A819927880F991F14
:1004D000FC01E055FF4F808191811D82281739076B
:1004E00011F081E08D8389818F5F89839D819923BC
:1004F00019F01C821B820AC08A818F5F8A838A81DD
:100500008530D0F281E090E09C838B838B819C814D
:1005100025960FB6F894DEBF0FBECDBFDF91CF9109
:100520000895CF93DF93CDB7DEB725970FB6F89434
:10053000DEBF0FBECDBF19821A821DC089819927E7
:10054000FC01E45CFD4F20818A819927FC01E45481
:10055000FF4F80811D82281711F081E08D838981F2
:100560008F5F89839D81992319F01C821B820AC0A9
:100570008A818F5F8A838A818B3001F781E090E0E6
:100580009C838B838B819C8125960FB6F894DEBF6C
:100590000FBECDBFDF91CF910895CF93DF93CDB73D
:1005A000DEB727970FB6F894DEBF0FBECDBF9C8392
:1005B0008B8319821A8220C089819927FC01E45C0F
:1005C000FD4F40818A8199279C018B819C81F90193
:1005D000E80FF91F80811F82481711F081E08F8397
:1005E00089818F5F89839F81992319F01E821D82E3
:1005F0000AC08A818F5F8A838A818930E9F681E027
:1006000090E09E838D838D819E8127960FB6F8940E
:10061000DEBF0FBECDBFDF91CF910895CF93DF93A3
:10062000CDB7DEB784ED90E00E94F3008FEF9FEF2F
:10063000A0E0B0E080936F0490937004A0937104E5
:10064000B093720480916F0490917004A091710432
:10065000B09172040197A109B10980936F0490933E
:100660007004A0937104B093720480916F04909110
:100670007004A0917104B09172040097A105B105B6
:1006800009F70E9483030097D9F110923402109267
:10069000330289ED90E00E94F3008FEF9FEFA0E01E
:1006A000B0E080936F0490937004A0937104B093B2
:1006B000720480916F0490917004A0917104B091C4
:1006C00072040197A109B10980936F04909370049B
:1006D000A0937104B093720480916F0490917004A0
:1006E000A0917104B09172040097A105B10509F7BA
:1006F0000E948303009721F010923402109233027B
:10070000DF91CF9108951F93CF93DF93CDB7DEB7DD
:1007100029970FB6F894DEBF0FBECDBF1C821B8297
:100720001A8219828FE48D838BE48E8360EA76E8E7
:1007300081E090E00E9443018A3031F080913302E1
:1007400090913402009791F380913302909134029A
:10075000009741F01986188632C089819A810196E6
:100760009A8389832B813C81CE010596FC01E20F9F
:10077000F31F108160EA76E881E090E00E94430177
:100780001F82181711F481E08F838B819C81019661
:100790009C838B839F81992301F760EA76E881E04F
:1007A00090E00E9443018A3031F0809133029091B1
:1007B0003402009791F389819A8199878887888587
:1007C000998529960FB6F894DEBF0FBECDBFDF9195
:1007D000CF911F910895CF93DF93CDB7DEB72697C2
:1007E0000FB6F894DEBF0FBECDBF10923402109248
:1007F00033021C821B821A82198260EA76E881E049
:1008000090E00E9443018A3031F080913302909150
:100810003402009791F38091330290913402009753
:1008200069F460EA76E881E090E00E9443018093F9
:100830007304809173048B3221F008C01E821D82E4
:1008400009C089819A8101969A83898389819A81D5
:100850009E838D838D819E8126960FB6F894DEBF90
:100860000FBECDBFDF91CF9108951F93CF93DF933C
:10087000CDB7DEB725970FB6F894DEBF0FBECDBF5C
:100880001C821B821A821982109234021092330247
:1008900060EA76E881E090E00E9443018A3061F0EE
:1008A0008091330290913402009791F305C08981C1
:1008B0009A8101969A8389838B819C81FC01E456FD
:1008C000FF4F108160EA76E881E090E00E944301EA
:1008D0001D82181711F481E08D838B819C81019614
:1008E0009C838B8381E09D818927882331F48091CB
:1008F0003302909134020097D1F260EA76E881E009
:1009000090E00E9443018A3031F08091330290914F
:100910003402009791F325960FB6F894DEBF0FBE10
:10092000CDBFDF91CF911F9108951F93CF93DF9398
:10093000CDB7DEB728970FB6F894DEBF0FBECDBF98
:100940001E821D821C821B821A82198260EA76E84E
:1009500081E090E00E9443018A3009F454C0809104
:10096000330290913402009789F34DC080919A022E
:1009700090919B02009709F45CC060EA76E881E000
:1009800090E00E944301809373048D819E81FC015D
:10099000EA55FF4F9081809173049817A1F58D81DE
:1009A0009E8101969E838D838D819E81FC01EA55F7
:1009B000FF4F108160EA76E881E090E00E944301F9
:1009C0001817F9F489819A8101969A83898305C061
:1009D0008B819C8101969C838B838D819E81019666
:1009E0009E838D838D819E81FC01EA55FF4F10818E
:1009F00060EA76E881E090E00E944301181741F335
:100A000002C01E821D8289819A81009709F4AECFAF
:100A100060EA76E881E090E00E9443018A30C1F705
:100A2000109234021092330289819A8198878F83C1
:100A300001C002C08F81988528960FB6F894DEBF5A
:100A40000FBECDBFDF91CF911F910895CF93DF935C
:100A5000CDB7DEB724970FB6F894DEBF0FBECDBF7B
:100A600069837A838B839C8389819A81AB81BC81E2
:100A70000197A109B10989839A83AB83BC838981DA
:100A80009A81AB81BC810097A105B10569F72496D5
:100A90000FB6F894DEBF0FBECDBFDF91CF910895A2
:100AA000CF93DF93CDB7DEB7A4E3B0E0E4E3F0E0AB
:100AB000808180688C93A5E3B0E0E5E3F0E090816D
:100AC00080E889278C93DF91CF910895CF93DF93AE
:100AD000CDB7DEB7A4E3B0E0E4E3F0E08081806866
:100AE0008C93A5E3B0E0E5E3F0E0808180688C932F
:100AF000DF91CF910895CF93DF93CDB7DEB7A4E315
:100B0000B0E0E4E3F0E0808180648C93A5E3B0E0A2
:100B1000E5E3F0E0908180E489278C93DF91CF9129
:100B20000895CF93DF93CDB7DEB7A4E3B0E0E4E35D
:100B3000F0E0808180648C93A5E3B0E0E5E3F0E031
:100B4000808180648C93DF91CF910895CF93DF9360
:100B5000CDB7DEB7A1E3B0E0E1E3F0E080818068EB
:100B60008C93A2E3B0E0E2E3F0E0908180E8892793
:100B70008C93DF91CF910895CF93DF93CDB7DEB7FC
:100B80002E970FB6F894DEBF0FBECDBF9E878D8720
:100B90004EC080E090E0A0E8BFE38B839C83AD83F0
:100BA000BE8326E636E646EE54E46B817C818D8179
:100BB0009E810E94B213DC01CB0189879A87AB87A3
:100BC000BC8720E030E040E85FE369857A858B856B
:100BD0009C850E943C1588230CF005C081E090E0C4
:100BE00098878F831AC020E03FEF4FE757E469856D
:100BF0007A858B859C850E94D01418160CF003C052
:100C000018861F820AC069857A858B859C850E941B
:100C10000112DC01CB0198878F838F8198859A839D
:100C2000898389819A810197F1F79A8389838D85D8
:100C30009E8501979E878D878D859E852FEF8F3F9F
:100C4000920709F0A6CF2E960FB6F894DEBF0FBE1E
:100C5000CDBFDF91CF910895CF93DF93CDB7DEB7AE
:100C6000CC5AD0400FB6F894DEBF0FBECDBF1A826B
:100C70001982E6E3F0E080819927817090708823E3
:100C800031F18CEA92E09C838B83E3EEF0E0FE830B
:100C9000ED83F7E0FF83ED81FE8100808D819E81F1
:100CA00001969E838D83EB81FC8100828B819C81E8
:100CB00001969C838B839F8191509F83EF81EE23CC
:100CC00051F789819A8106969A83898325C08CEA97
:100CD00092E099878887EAEEF0E0FB87EA87F7E001
:100CE000FC87EA85FB8500808A859B8501969B872A
:100CF0008A87E885F9850082888599850196998794
:100D000088879C8591509C87EC85EE2351F78981DB
:100D10009A8106969A838983E0E3F0E0808199279F
:100D200084709070009741F189819A8184559D4F1C
:100D30009E878D8781EF90E0988B8F8797E0998BC6
:100D4000EF85F88900808F8598890196988B8F8729
:100D5000ED85FE8500828D859E8501969E878D8717
:100D600099899150998BE989EE2351F789819A816C
:100D700006969A83898327C089819A8184559D4FDD
:100D80009B8B8A8B88EF90E09D8B8C8B97E09E8B62
:100D9000EC89FD8900808C899D8901969D8B8C8BC7
:100DA000EA89FB8900828A899B8901969B8B8A8BC1
:100DB0009E8991509E8BEE89EE2351F789819A810D
:100DC00006969A838983E5E3F0E08081882344F5E1
:100DD00089819A8184559D4F988F8F8B8FEF90E0FA
:100DE0009A8F898F9AE09B8FE98DFA8D0080898D8B
:100DF0009A8D01969A8F898FEF89F88D00828F895D
:100E0000988D0196988F8F8B9B8D91509B8FEB8D3A
:100E1000EE2351F789819A8109969A83898327C0A5
:100E200089819A8184559D4F9D8F8C8F89E091E0B7
:100E30009F8F8E8F9AE098A3EE8DFF8D00808E8D10
:100E40009F8D01969F8F8E8FEC8DFD8D00828C8DF6
:100E50009D8D01969D8F8C8F98A1915098A3E8A1AC
:100E6000EE2351F789819A8109969A838983E5E374
:100E7000F0E08081992780749070009741F189811A
:100E80009A8184559D4F9AA389A383E191E09CA305
:100E90008BA39AE09DA3EBA1FCA100808BA19CA158
:100EA00001969CA38BA3E9A1FAA1008289A19AA132
:100EB00001969AA389A39DA191509DA3EDA1EE2334
:100EC00051F789819A8109969A83898327C08981FC
:100ED0009A8184559D4F9FA38EA38DE191E099A7A0
:100EE00088A79AE09AA7E8A5F9A5008088A599A502
:100EF000019699A788A7EEA1FFA100828EA19FA1CC
:100F000001969FA38EA39AA591509AA7EAA5EE23D6
:100F100051F789819A8109969A838983E9E3F0E000
:100F20008081992784709070009741F189819A811E
:100F300084559D4F9CA78BA787E291E09EA78DA724
:100F400099E09FA7EDA5FEA500808DA59EA5019621
:100F50009EA78DA7EBA5FCA500828BA59CA501965D
:100F60009CA78BA79FA591509FA7EFA5EE2351F7B4
:100F700089819A8108969A83898327C089819A8179
:100F800084559D4F99AB88AB80E391E09BAB8AABD6
:100F900099E09CABEAA9FBA900808AA99BA90196CC
:100FA0009BAB8AABE8A9F9A9008288A999A9019607
:100FB00099AB88AB9CA991509CABECA9EE2351F75F
:100FC00089819A8108969A838983E9E3F0E0808198
:100FD000992782709070009741F189819A81845598
:100FE0009D4F9EAB8DAB89E391E098AF8FAB99E0BD
:100FF00099AFEFA9F8AD00808FA998AD019698AF91
:101000008FABEDA9FEA900828DA99EA901969EAB8A
:101010008DAB99AD915099AFE9ADEE2351F7898130
:101020009A8108969A83898327C089819A818455F9
:101030009D4F9BAF8AAF82E491E09DAF8CAF99E06A
:101040009EAFECADFDAD00808CAD9DAD01969DAF2A
:101050008CAFEAADFBAD00828AAD9BAD01969BAF34
:101060008AAF9EAD91509EAFEEADEE2351F78981D0
:101070009A8108969A838983E9E3F0E08081992731
:1010800081709070882309F440C089819A818455C9
:101090009D4F21969FAF8EAF21978BE491E02396D1
:1010A0009FAF8EAF239799E024969FAF2497239606
:1010B000EEADFFAD2397008023968EAD9FAD2397B5
:1010C000019623969FAF8EAF23972196EEADFFAD8D
:1010D0002197008221968EAD9FAD21970196219692
:1010E0009FAF8EAF219724969FAD24979150249661
:1010F0009FAF24972496EFAD2497EE23C1F6898104
:101100009A8108969A8389833FC089819A81845500
:101110009D4F26969FAF8EAF269784E591E0289647
:101120009FAF8EAF289799E029969FAF2997289671
:10113000EEADFFAD2897008028968EAD9FAD289725
:10114000019628969FAF8EAF28972696EEADFFADFD
:101150002697008226968EAD9FAD269701962696FD
:101160009FAF8EAF269729969FAD299791502996CC
:101170009FAF29972996EFAD2997EE23C1F6898174
:101180009A8108969A838983E6E3F0E08081882338
:101190000CF040C089819A8184559D4F2B969FAF5A
:1011A0008EAF2B978DE591E02D969FAF8EAF2D974B
:1011B00099E02E969FAF2E972D96EEADFFAD2D9711
:1011C00000802D968EAD9FAD2D9701962D969FAFE9
:1011D0008EAF2D972B96EEADFFAD2B9700822B9601
:1011E0008EAD9FAD2B9701962B969FAF8EAF2B9711
:1011F0002E969FAD2E9791502E969FAF2E972E969E
:10120000EFAD2E97EE23C1F689819A8108969A83D5
:1012100089833FC089819A8184559D4F60969FAF95
:101220008EAF609786E691E062969FAF8EAF629731
:1012300099E063969FAF63976296EEADFFAD6297BC
:10124000008062968EAD9FAD6297019662969FAFC9
:101250008EAF62976096EEADFFAD609700826096AC
:101260008EAD9FAD6097019660969FAF8EAF6097F1
:1012700063969FAD6397915063969FAF6397639614
:10128000EFAD6397EE23C1F689819A8108969A8320
:101290008983E6E3F0E0808199278074907000975D
:1012A00009F440C089819A8184559D4F65969FAF0E
:1012B0008EAF65978FE691E067969FAF8EAF679789
:1012C00099E068969FAF68976796EEADFFAD679718
:1012D000008067968EAD9FAD6797019667969FAF2A
:1012E0008EAF67976596EEADFFAD65970082659608
:1012F0008EAD9FAD6597019665969FAF8EAF659752
:1013000068969FAD6897915068969FAF689768966A
:10131000EFAD6897EE23C1F689819A8108969A838A
:1013200089833FC089819A8184559D4F6A969FAF7A
:101330008EAF6A9788E791E06C969FAF8EAF6C97FF
:1013400099E06D969FAF6D976C96EEADFFAD6C9783
:1013500000806C968EAD9FAD6C9701966C969FAF9A
:101360008EAF6C976A96EEADFFAD6A9700826A9673
:101370008EAD9FAD6A9701966A969FAF8EAF6A97C2
:101380006D969FAD6D9791506D969FAF6D976D96D1
:10139000EFAD6D97EE23C1F689819A8108969A8305
:1013A0008983E6E3F0E0808199278072907000974E
:1013B00009F440C089819A8184559D4F6F969FAFF3
:1013C0008EAF6F9781E891E0A1969FAF8EAFA19706
:1013D00099E0A2969FAFA297A196EEADFFADA1971F
:1013E0000080A1968EAD9FADA1970196A1969FAF6B
:1013F0008EAFA1976F96EEADFFAD6F9700826F969F
:101400008EAD9FAD6F9701966F969FAF8EAF6F9722
:10141000A2969FADA2979150A2969FAFA297A29637
:10142000EFADA297EE23C1F689819A8108969A833F
:1014300089833FC089819A8184559D4FA4969FAF2F
:101440008EAFA4978AE891E0A6969FAF8EAFA6973D
:1014500099E0A7969FAFA797A696EEADFFADA6978A
:101460000080A6968EAD9FADA6970196A6969FAFDB
:101470008EAFA697A496EEADFFADA4970082A4967A
:101480008EAD9FADA4970196A4969FAF8EAFA49703
:10149000A7969FADA7979150A7969FAFA797A7969E
:1014A000EFADA797EE23C1F689819A8108969A83BA
:1014B0008983E6E3F0E0808199278072907000973D
:1014C00009F440C089819A8184559D4FA9969FAFA8
:1014D0008EAFA99781E891E0AB969FAF8EAFAB97A7
:1014E00099E0AC969FAFAC97AB96EEADFFADAB97E6
:1014F0000080AB968EAD9FADAB970196AB969FAF3C
:101500008EAFAB97A996EEADFFADA9970082A996D5
:101510008EAD9FADA9970196A9969FAF8EAFA99763
:10152000AC969FADAC979150AC969FAFAC97AC96F4
:10153000EFADAC97EE23C1F689819A8108969A8324
:1015400089833FC089819A8184559D4FAE969FAF14
:101550008EAFAE978AE891E0E0969FAF8EAFE097AE
:1015600099E0E1969FAFE197E096EEADFFADE09791
:101570000080E0968EAD9FADE0970196E0969FAF1C
:101580008EAFE097AE96EEADFFADAE970082AE9611
:101590008EAD9FADAE970196AE969FAF8EAFAE97D4
:1015A000E1969FADE1979150E1969FAFE197E1966B
:1015B000EFADE197EE23C1F689819A8108969A836F
:1015C0008983E6E3F0E0808199278071907000972D
:1015D00009F440C089819A8184559D4FE3969FAF5D
:1015E0008EAFE39783E991E0E5969FAF8EAFE597E5
:1015F00099E0E6969FAFE697E596EEADFFADE597ED
:101600000080E5968EAD9FADE5970196E5969FAF7C
:101610008EAFE597E396EEADFFADE3970082E396DC
:101620008EAD9FADE3970196E3969FAF8EAFE397A4
:10163000E6969FADE6979150E6969FAFE697E696C1
:10164000EFADE697EE23C1F689819A8108969A83D9
:1016500089833FC089819A8184559D4FE8969FAFC9
:101660008EAFE8978CE991E0EA969FAF8EAFEA974C
:1016700099E0EB969FAFEB97EA96EEADFFADEA9758
:101680000080EA968EAD9FADEA970196EA969FAFED
:101690008EAFEA97E896EEADFFADE8970082E89648
:1016A0008EAD9FADE8970196E8969FAF8EAFE89715
:1016B000EB969FADEB979150EB969FAFEB97EB9628
:1016C000EFADEB97EE23C1F689819A8108969A8354
:1016D0008983E6E3F0E08081992788709070009715
:1016E00009F448C089819A8184559D4FED969FAF3A
:1016F0008EAFED9785EA91E0EF969FAF8EAFEF97B3
:1017000099E0C158DF4F9883CF57D040EF96EEADA8
:10171000FFADEF970080EF968EAD9FADEF970196EE
:10172000EF969FAF8EAFEF97ED96EEADFFADED97D5
:101730000082ED968EAD9FADED970196ED969FAF31
:101740008EAFED97C158DF4F9881CF57D040915061
:10175000C158DF4F9883CF57D040C158DF4FE88141
:10176000CF57D040EE2391F689819A8108969A83CB
:10177000898357C089819A8184559D4FC058DF4F16
:1017800099838883C058D0408EEA91E0CE57DF4FCE
:1017900099838883C258D04099E0CC57DF4F988313
:1017A000C458D040CE57DF4FE881F981C258D040AD
:1017B0000080CE57DF4F88819981C258D040019672
:1017C000CE57DF4F99838883C258D040C058DF4F2F
:1017D000E881F981C058D0400082C058DF4F88812D
:1017E0009981C058D0400196C058DF4F99838883B3
:1017F000C058D040CC57DF4F9881C458D04091504A
:10180000CC57DF4F9883C458D040CC57DF4FE88186
:10181000C458D040EE2331F689819A8108969A8384
:101820008983E6E3F0E080819927847090700097C7
:1018300009F458C089819A8184559D4FCB57DF4F59
:1018400099838883C558D04087EB91E0C957DF4F13
:1018500099838883C758D04099E0C757DF4F988352
:10186000C958D040C957DF4FE881F981C758D040E7
:101870000080C957DF4F88819981C758D0400196B1
:10188000C957DF4F99838883C758D040CB57DF4F64
:10189000E881F981C558D0400082CB57DF4F88815D
:1018A0009981C558D0400196CB57DF4F99838883E3
:1018B000C558D040C757DF4F9881C958D040915084
:1018C000C757DF4F9883C958D040C757DF4FE881CB
:1018D000C958D040EE2331F689819A8108969A83BF
:1018E000898357C089819A8184559D4FC657DF4FA0
:1018F00099838883CA58D04080EC91E0C457DF4F69
:1019000099838883CC58D04099E0C257DF4F9883A1
:10191000CE58D040C457DF4FE881F981CC58D04031
:101920000080C457DF4F88819981CC58D040019600
:10193000C457DF4F99838883CC58D040C657DF4FB8
:10194000E881F981CA58D0400082C657DF4F8881AC
:101950009981CA58D0400196C657DF4F9983888332
:10196000CA58D040C257DF4F9881CE58D0409150CE
:10197000C257DF4F9883CE58D040C257DF4FE8811F
:10198000CE58D040EE2331F689819A8108969A8309
:101990008983E6E3F0E08081992782709070009758
:1019A00009F458C089819A8184559D4FC157DF4FF2
:1019B00099838883CF58D04089EC91E0CF56DF4F90
:1019C00099838883C159D04099E0CD56DF4F9883E1
:1019D000C359D040CF56DF4FE881F981C159D0407B
:1019E0000080CF56DF4F88819981C159D040019640
:1019F000CF56DF4F99838883C159D040C157DF4FFD
:101A0000E881F981CF58D0400082C157DF4F8881EB
:101A10009981CF58D0400196C157DF4F9983888371
:101A2000CF58D040CD56DF4F9881C359D040915008
:101A3000CD56DF4F9883C359D040CD56DF4FE88154
:101A4000C359D040EE2331F689819A8108969A8352
:101A5000898357C089819A8184559D4FCC56DF4F29
:101A600099838883C459D04082ED91E0CA56DF4FF4
:101A700099838883C659D04099E0C856DF4F988330
:101A8000C859D040CA56DF4FE881F981C659D040C5
:101A90000080CA56DF4F88819981C659D04001968F
:101AA000CA56DF4F99838883C659D040CC56DF4F42
:101AB000E881F981C459D0400082CC56DF4F88813B
:101AC0009981C459D0400196CC56DF4F99838883C1
:101AD000C459D040C856DF4F9881C859D040915062
:101AE000C856DF4F9883C859D040C856DF4FE881A9
:101AF000C859D040EE2331F689819A8108969A839D
:101B00008983E6E3F0E080819927817090708823D3
:101B100009F458C089819A8184559D4FC756DF4F7B
:101B200099838883C959D0408BED91E0C556DF4F2A
:101B300099838883CB59D04099E0C356DF4F98836F
:101B4000CD59D040C556DF4FE881F981CB59D040FF
:101B50000080C556DF4F88819981CB59D0400196CE
:101B6000C556DF4F99838883CB59D040C756DF4F86
:101B7000E881F981C959D0400082C756DF4F88817A
:101B80009981C959D0400196C756DF4F9983888300
:101B9000C959D040C356DF4F9881CD59D04091509C
:101BA000C356DF4F9883CD59D040C356DF4FE881ED
:101BB000CD59D040EE2331F689819A8108969A83D7
:101BC000898357C089819A8184559D4FC256DF4FC2
:101BD00099838883CE59D04084EE91E0C056DF4F80
:101BE00099838883C05AD04099E0CE55DF4F9883BF
:101BF000C25AD040C056DF4FE881F981C05AD04068
:101C00000080C056DF4F88819981C05AD04001962C
:101C1000C056DF4F99838883C05AD040C256DF4FE9
:101C2000E881F981CE59D0400082C256DF4F8881C9
:101C30009981CE59D0400196C256DF4F998388834F
:101C4000CE59D040CE55DF4F9881C25AD0409150E6
:101C5000CE55DF4F9883C25AD040CE55DF4FE88132
:101C6000C25AD040EE2331F689819A8108969A8330
:101C70008983E0E3F0E08081992788709070009775
:101C800009F458C089819A8184559D4FCD55DF4F05
:101C900099838883C35AD0408DEE91E0CB55DF4FB6
:101CA00099838883C55AD04097E0C955DF4F988300
:101CB000C75AD040CB55DF4FE881F981C55AD04093
:101CC0000080CB55DF4F88819981C55AD04001965D
:101CD000CB55DF4F99838883C55AD040CD55DF4F10
:101CE000E881F981C35AD0400082CD55DF4F888109
:101CF0009981C35AD0400196CD55DF4F998388838F
:101D0000C35AD040C955DF4F9881C75AD04091502F
:101D1000C955DF4F9883C75AD040C955DF4FE88176
:101D2000C75AD040EE2331F689819A8106969A836C
:101D3000898357C089819A8184559D4FC855DF4F4B
:101D400099838883C85AD04084EF91E0C655DF4F0D
:101D500099838883CA5AD04097E0C455DF4F98834F
:101D6000CC5AD040C655DF4FE881F981CA5AD040DD
:101D70000080C655DF4F88819981CA5AD0400196AC
:101D8000C655DF4F99838883CA5AD040C855DF4F64
:101D9000E881F981C85AD0400082C855DF4F888158
:101DA0009981C85AD0400196C855DF4F99838883DE
:101DB000C85AD040C455DF4F9881CC5AD04091507A
:101DC000C455DF4F9883CC5AD040C455DF4FE881CB
:101DD000CC5AD040EE2331F689819A8106969A83B7
:101DE0008983C455DF4F0FB6F894DEBF0FBECDBF59
:101DF000DF91CF910895CF93DF93CDB7DEB72B97C7
:101E00000FB6F894DEBF0FBECDBF9C838B838AE0F4
:101E100090E09A83898389819A81ECE7F2E028EC4B
:101E200030E0AC01B901CF010E940A1889819A8182
:101E300084589D4F98878F838CE992E09A87898791
:101E40009FE09B87E985FA85008089859A850196C0
:101E50009A878987EF81F88500828F81988501961E
:101E600098878F839B8591509B87EB85EE2351F755
:101E700089819A810C969A83898389819A81FC0150
:101E8000E458FD4F82E2808389819A8101969A838A
:101E9000898389819A81FC01E458FD4F10828CE787
:101EA00092E00E94F3008FEF9FEFA0E0B0E08093FC
:101EB0006F0490937004A0937104B09372048091A6
:101EC0006F0490917004A0917104B0917204019715
:101ED000A109B10980936F0490937004A0937104D9
:101EE000B093720480916F0490917004A09171047A
:101EF000B09172040097A105B10509F780915204D1
:101F000090915304009789F008C060EA76E881E078
:101F100090E00E94430180937304809173048E3398
:101F2000A1F78B819C810E941B01109234021092B8
:101F300033020E94EB03009719F41E821D8237C002
:101F4000109234021092330260EA76E881E090E069
:101F50000E9443018093730480914C0390914D0340
:101F600090934D0380934C03809173048A3061F702
:101F700010923402109233020E948303009719F4E6
:101F80001E821D8214C010923402109233028FEF11
:101F90009FEFA0E0B0E080936F0490937004A09353
:101FA0007104B093720481E090E09E838D838D81F3
:101FB0009E812B960FB6F894DEBF0FBECDBFDF918A
:101FC000CF910895CF93DF93CDB7DEB76F970FB65C
:101FD000F894DEBF0FBECDBF1092AB021092790411
:101FE000109278041A8219821C821B821E821D8222
:101FF0000DC02D813E818BEF91E0F901E455FD4F3D
:1020000080838D819E8101969E838D838D819E81AB
:10201000803A910574F30E94490084E190E0A1E0C8
:10202000B0E080936F0490937004A0937104B09318
:10203000720480916F0490917004A0917104B0912A
:1020400072040197A109B10980936F049093700401
:10205000A0937104B093720480916F049091700406
:10206000A0917104B09172040097A105B10509F720
:10207000EAE3F0E084E0808360E673EE86E190E0DE
:102080000E942605ABE3B0E0EBE3F0E090818BEF3C
:1020900089238C93AAE3B0E0EAE3F0E090818BEF30
:1020A00089238C9380915204909153040097D1F32B
:1020B0000E9495040E940E0300C0809152049091EA
:1020C00053040097D1F31092AB021C821B820E9432
:1020D000EB03009709F450C1EFE4F0E0108260EAEE
:1020E00076E881E090E00E94430180937304809140
:1020F00073048D3031F1809173048A3011F1309185
:10210000AB02832F992720917304FC01E45CFD4FFF
:102110002083832F8F5F8093AB0280917304992774
:10212000C0978A30910568F48B819C81209173045B
:10213000FC01E85AFB4F20838B819C8101969C8394
:102140008B83809173048A3051F61092340210927E
:10215000330288E594E00E94EC179A838983898191
:102160009A819F938F938CEF91E09F938F9382E658
:1021700094E09F938F930E941B188DB79EB706968D
:102180000FB6F8949EBF0FBE8DBF0E9491028823A8
:1021900009F493CF82E694E00E94F3008FEF9FEF63
:1021A000A0E0B0E080936F0490937004A09371045A
:1021B000B093720480916F0490917004A0917104A7
:1021C000B09172040197A109B10980936F049093B3
:1021D0007004A0937104B093720480916F04909185
:1021E0007004A0917104B09172040097A105B1052B
:1021F00009F70E94EB031092AB0210922E0210928C
:102200002D0260EA76E881E090E00E94430180932D
:10221000730480917304823249F480912D0290916D
:102220002E02019690932E0280932D0280912D0212
:1022300090912E0283309105A9F48091730499271F
:10224000C0978A30910570F43091AB02832F9927A3
:1022500020917304FC01E456FD4F2083832F8F5F90
:102260008093AB0280914C0390914D0390934D036A
:1022700080934C03809173048A3019F68091AB02ED
:102280009927FC01E456FD4F1082109234021092FF
:1022900033021092AB0260EA76E881E090E00E949F
:1022A000430180937304809173048D3091F0809189
:1022B00073048A3071F03091AB02832F99272091FB
:1022C0007304FC01E45CFD4F2083832F8F5F8093B8
:1022D000AB02809173048A30F1F6109234021092AE
:1022E00033020E94830310923402109233028AE771
:1022F00090E00E94CD02813099F40E9466050E9410
:102300002C06E5E3F0E0808188232CF48CEA92E04F
:102310000E94FB0ED2CE87E092E00E94FB0ECDCE53
:102320008CE890E00E94CD028130B1F40E949105CA
:102330000E942C06E5E3F0E080819927807490707C
:10234000009729F08CEA92E00E94FB0EB6CE87E05F
:1023500092E00E94FB0EB1CE88E690E00E94CD0292
:10236000813009F0AACE0E94A6050E942C068CEAB4
:1023700092E00E94FB0EA1CE1092AB023091AB0214
:10238000832F992720917304FC01E45CFD4F208387
:10239000832F8F5F8093AB0260EA76E881E090E064
:1023A0000E94430180937304809173048A3071F01A
:1023B0003091AB02832F992720917304FC01E45CD8
:1023C000FD4F2083832F8F5F8093AB028091730436
:1023D0008A3011F710923402109233021092AB023D
:1023E000EFE4F0E010820E944F02882309F465CEEA
:1023F000AFE4B0E0EFE4F0E0908180E189278C93D6
:102400005CCEEF92FF920F931F937B018C0120E033
:1024100030E040E05FE40E94061588237CF020E075
:1024200030E040E05FE4C801B7010E9454130E940D
:102430007215605070408040904804C0C801B701D8
:102440000E9472151F910F91FF90EF900895A0E0E8
:10245000B0E0EDE2F2E10C94681BFC016A019081AE
:10246000923008F41BC1DB018C91823080F09430F3
:1024700061F4843009F012C19181EB0189819817D0
:1024800009F40CC1E1E2F2E009C1843011F4FB016E
:1024900005C1823091F4923009F000C1EA01DF01F8
:1024A00088E00D9009928150E1F78181FB019181D3
:1024B0008923E6018983F601F1C0923041F36280FD
:1024C0007380EB018A809B80E480F5800681178110
:1024D0002C813D814E815F815301A818B908C50147
:1024E000B7FCABC080970CF457C0861497040CF46B
:1024F000BEC03401EE24FF2487019181FB0181815C
:10250000981709F4A6C0992309F49CC02E193F0915
:10251000400B510B57FDB0C0E60119827B826A82E5
:10252000F6012483358346835783E6012C813D8160
:102530004E815F8179018A01DA01C9010197A10900
:10254000B1098F5F9F4FAF4FBF43F8F4E6016A8137
:102550007B81A8019701220F331F441F551F615033
:10256000704079018A01DA01C9010197A109B10915
:102570008F5F9F4FAF4FBF4360F3E6017B836A835A
:10258000F601248335834683578383E0D6018C93F9
:1025900057FD39C0F60182C086149704B4F4C0E038
:1025A000D0E0DA01C90181709070A070B0705695CA
:1025B000479537952795282B392B4A2B5B2B21964E
:1025C000AC16BD0671F78A0C9B1C681479040CF0DC
:1025D00094CFC0E0D0E05401A618B708D801C701D5
:1025E00081709070A070B07016950795F794E7947D
:1025F000E82AF92A0A2B1B2B2196AC16BD0671F787
:102600006A0C7B1C7ACFDA01C901B695A79597951C
:1026100087952170307040705070282B392B4A2BD1
:102620005B2BE6012C833D834E835F838A819B81F4
:1026300001969B838A83F60131C0882799278A19DE
:102640009B0950CFE21AF30A040B150BA80197015E
:1026500061CFE60199837B826A822E0D3F1D401F68
:10266000511FF60124833583468357838ECF20E0A4
:1026700030E040E050E041CF81E0E60189837B8299
:102680006A8250954095309521953F4F4F4F5F4F4F
:10269000F601248335834683578347CFCF01EEE08D
:1026A000CDB7DEB70C94841BA0E2B0E0EAE5F3E11D
:1026B0000C94701B69837A838B839C832D833E8368
:1026C0004F83588789E1E82EF12CEC0EFD1EB701EF
:1026D000CE0101960E94E4168E010F5E1F4FB801D5
:1026E000CE0105960E94E4168A8991E089278A8B9B
:1026F000AE01475F5F4FB801C7010E9427120E94D9
:10270000C215E6E0A0960C948C1BA0E2B0E0EBE8CA
:10271000F3E10C94701B69837A838B839C832D83F4
:102720003E834F83588799E1E92EF12CEC0EFD1E74
:10273000B701CE0101960E94E4168E010F5E1F4F75
:10274000B801CE0105960E94E416AE01475F5F4FC7
:10275000B801C7010E9427120E94C215E6E0A096A8
:102760000C948C1BA0E2B0E0E8EBF3E10C94641B4A
:1027700069837A838B839C832D833E834F83588721
:102780008E01075E1F4FB801CE0101960E94E4162C
:10279000F1E1EF2EF12CEC0EFD1EB701CE010596F6
:1027A0000E94E416898D823078F09989923040F445
:1027B00020E09A8D8A89981321E02A8BB701E9C01D
:1027C000843051F4923061F020E09A8D8A89981318
:1027D00021E02A8FB801DDC0943029F4823041F71E
:1027E00061E272E0D6C0823079F3923009F32D8D28
:1027F0003E8D4F8D58A18D899E89AF89B88D222439
:1028000033242101AA24BB246501EE24FF2487017F
:1028100060E070E00DC06F5F7F4F6032710599F12D
:10282000880F991FAA1FBB1F569547953795279567
:1028300020FF19C0280E391E4A1E5B1E662477240D
:102840004301281639064A065B0628F4E1E06E2E9D
:10285000712C812C912CAE0CBF1CC01ED11EA60C5D
:10286000B71CC81CD91CEE0CFF1C001F111FB7FFA2
:10287000D2CFE1E06E2E712C812C912CE628F72826
:1028800008291929C8CF8B8D9C8D2B893C89820FF3
:10289000931F02969C878B871A869A8D8A89981730
:1028A00011F081E08A87D7FE17C08B859C85A0FE3A
:1028B0000CC0569447943794279420E030E040E0D1
:1028C00050E8222A332A442A552AD694C794B7942A
:1028D000A79401969C878B8730E0A31630E0B3065F
:1028E00030E0C30630E4D30618F58B859C850EC016
:1028F000220C331C441C551C019720E0A21620E03A
:10290000B20620E0C20620E4D20680F4AA0CBB1C6A
:10291000CC1CDD1C57FEECCF31E0632E712C812CDA
:10292000912CA628B728C828D928E2CF9C878B8766
:10293000D601C5018F779070A070B070803491057A
:10294000A105B10551F0AD86BE86CF86D88A83E059
:102950008987BE01675F7F4F1CC0A7FCF4CF21149D
:1029600031044104510479F380E490E0A0E0B0E048
:10297000A80EB91ECA1EDB1E80E8682E8FEF782EC7
:102980008FEF882E8FEF982EA620B720C820D92051
:10299000DACFCB010E94C215E2E1A0960C94801B15
:1029A000A8E1B0E0E6EDF4E10C94701B69837A8352
:1029B0008B839C832D833E834F83588781E1E82E50
:1029C000F12CEC0EFD1EB701CE0101960E94E4161B
:1029D0008E01075F1F4FB801CE0105960E94E416D5
:1029E0008989823018F42FEF3FEF0BC08985823040
:1029F000D0F3B801C7010E948317282F332727FD82
:102A00003095C901E6E068960C948C1BA8E1B0E013
:102A1000ECE0F5E10C94701B69837A838B839C83D3
:102A20002D833E834F83588781E1E82EF12CEC0EF5
:102A3000FD1EB701CE0101960E94E4168E01075FCC
:102A40001F4FB801CE0105960E94E4168989823095
:102A500018F42FEF3FEF0BC089858230D0F3B80117
:102A6000C7010E948317282F332727FD3095C901FE
:102A7000E6E068960C948C1BA8E1B0E0E2E4F5E196
:102A80000C94701B69837A838B839C832D833E8394
:102A90004F83588781E1E82EF12CEC0EFD1EB70123
:102AA000CE0101960E94E4168E01075F1F4FB80108
:102AB000CE0105960E94E4168989823018F0898536
:102AC000823018F421E030E008C0B801C7010E944C
:102AD0008317282F332727FD3095C901E6E0689634
:102AE0000C948C1BACE0B0E0E8E7F5E10C94741BAF
:102AF00069837A838B839C83BE016B5F7F4FCE019A
:102B000001960E94E4168D81823061F0823050F08F
:102B1000843069F48E81882359F52FEF3FEF4FEF12
:102B20005FE72AC020E030E040E050E025C02F8180
:102B3000388537FDF7CF2F31310564F78EE190E00E
:102B4000821B930B29853A854B855C8504C056957D
:102B50004795379527958A95D2F78E81882361F01E
:102B600050954095309521953F4F4F4F5F4F04C092
:102B700020E030E040E050E8CA01B901E2E02C96E4
:102B80000C94901B4F925F926F927F928F929F92C4
:102B9000AF92BF92DF92EF92FF920F931F9320E0CC
:102BA00030E040E050E0FC01E480F58006811781D0
:102BB000D1808081823038F4D801C701A061AF771D
:102BC000B0706FEFD9C0843009F46EC0823009F460
:102BD00071C0E114F1040105110509F46BC0828193
:102BE00093816FEF823896070CF06AC062E87FEF3E
:102BF000681B790B6A3171050CF080C047015801E0
:102C0000062E04C0B694A794979487940A94D2F79A
:102C100044245524320181E090E0A0E0B0E004C0FB
:102C2000880F991FAA1FBB1F6A95D2F70197A109A8
:102C3000B109E822F9220A231B23E114F10401055A
:102C4000110529F061E0462E512C612C712C850173
:102C50007401E428F52806291729D801C7018F77C0
:102C60009070A070B07080349105A105B10509F491
:102C700057C0D801C701CF96A11DB11D60E070E01B
:102C80008030E0E09E07E0E0AE07E0E4BE0710F031
:102C900061E070E027E0B695A795979587952A950E
:102CA000D1F7AF77B07068C080E090E0A0E0B0E00E
:102CB0006FEF62C080E090E0A0E0B0E060E05CC058
:102CC000803891058CF7BC0161587F4FD801C7014E
:102CD0008F779070A070B07080349105A105B10518
:102CE000A1F08FE390E0A0E0B0E0E80EF91E0A1F2B
:102CF0001B1F17FD28C0D801C701CCCF60E070E0D2
:102D000080E090E0A0E0B0E0CCCFE7FEF2CF80E43E
:102D100090E0A0E0B0E0E80EF91E0A1F1B1FE9CF0B
:102D2000E7FC18C080E090E060E0E61660E0F606A0
:102D300060E0060760E4160710F081E090E0BC0157
:102D4000D801C701A7CF16950795F794E7946F5F51
:102D50007F4FD1CFD801C701805C9F4FAF4FBF4F8E
:102D600060E070E08030E0E09E07E0E0AE07E0E485
:102D7000BE0708F48FCF8CCF282F392F9A2F9F773B
:102D8000842F8078892B962F9795992797958F7701
:102D9000482F492B6695852F8078862BD794DD2484
:102DA000D7948F77582F5D29CA01B9011F910F91D0
:102DB000FF90EF90DF90BF90AF909F908F907F90AB
:102DC0006F905F904F900895FC01DB01208131816D
:102DD0009281492F4F7750E0991F9927991F83813E
:102DE000682F660F692B881F8827881FFD01818344
:102DF000662309F049C0211531054105510509F443
:102E000070C082E89FEFFD0193838283220F331FFE
:102E1000441F551F220F331F441F551F220F331FFE
:102E2000441F551F220F331F441F551F220F331FEE
:102E3000441F551F220F331F441F551F220F331FDE
:102E4000441F551F83E08C932030F0E03F07F0E0F3
:102E50004F07F0E45F0790F482E89FEF220F331FE3
:102E6000441F551F0197203060E0360760E0460799
:102E700060E4560798F3FD0193838283FD01248368
:102E800035834683578308956F3F71F1862F9927C5
:102E90008F579040FD019383828383E08C93220FB0
:102EA000331F441F551F220F331F441F551F220F6E
:102EB000331F441F551F220F331F441F551F220F5E
:102EC000331F441F551F220F331F441F551F220F4E
:102ED000331F441F551F5064248335834683578313
:102EE000089582E08C93089521153105410551051F
:102EF00019F484E08C93089544FD02C01C92BECF67
:102F000081E08C93BBCFEF92FF920F931F93CF93EF
:102F1000DF93FC01DB018081823050F09C91923084
:102F200038F0843041F49430B1F08181882381F409
:102F300061E070E04BC09430E9F18230A1F0923052
:102F4000A1F36181ED018981681791F0662381F316
:102F50006FEF7FEF3BC0EB018981682F772781817D
:102F6000681B710933C0923059F560E070E02EC0E3
:102F700022813381ED018A819B818217930734F38B
:102F8000281739079CF0E480F58006811781FD0140
:102F900024813581468157812E153F054007510711
:102FA000A8F2E216F30604071507F8F6662309F0FF
:102FB000BFCFCECFFB018181882309F0B9CFC8CF25
:102FC000EB018981882309F0B3CFC2CFCB01E6E0C2
:102FD000CDB7DEB70C948C1BFC0188279927E894A9
:102FE00021912032E9F3293010F02E30C8F32B3232
:102FF00041F02D3239F4689404C00E941318820FF6
:10300000911D219120532A30C0F31EF49095819593
:103010009F4F0895FB01DC0102C001900D924150C9
:103020005040D8F708957AE0979F902D879F802D84
:10303000910D112408950F931F93CF93DF93CDB774
:10304000DEB760970FB6F894DEBF0FBECDBF0F8915
:10305000188D86E08E831C830B838FEF9FE7988704
:103060008F83AE01455E5F4F5A834983698D7A8DA8
:10307000CE0103960E944D1829853A85020F131F31
:10308000F801108260960FB6F894DEBF0FBECDBF78
:10309000DF91CF911F910F9108952F923F924F9200
:1030A0005F926F927F928F929F92AF92BF92CF92D8
:1030B000DF92EF92FF920F931F93CF93DF93CDB7E1
:1030C000DEB764970FB6F894DEBF0FBECDBFCC2439
:1030D000DD2476011C017C8B6B8B2A01FC0117829D
:1030E0001682838181FD03C08FEF9FEF88C2AA24DF
:1030F000BB2472C2A0FE57C28A8980538A30E8F48A
:10310000FA89F03341F42D85222329F4A3FC03C06E
:1031100080E091E06FC08AE0ED85E802C0011124F3
:10312000FA89F80FF053FD87F7FF02C02FE72D87CC
:10313000A3FC4CC23D853E8749C2C5018870907092
:10314000A3FE05C0ED85EE2311F4F1E0FD872A8989
:10315000283624F525360CF05BC0233509F480C0F1
:1031600024358CF42B32C1F12C3234F42032C1F1ED
:10317000233209F00DC23CC03A893D32B1F13E32F2
:1031800009F006C23AC08A89833609F449C08436F8
:103190000CF081C0883509F0FBC11BC0EA89E0371B
:1031A00009F4A3C0E13744F4EC3669F1EF3671F06D
:1031B000E93609F0EDC16FC0FA89F53709F49DC011
:1031C000F83739F0F33709F0E3C134C028E0298B30
:1031D00094C030E1398B91C080E190E0A82AB92AEF
:1031E000E0E2F0E0AE2ABF2AF1C120E830E00DC0F5
:1031F00080E490E0A82AB92AE9C1E8E0F0E0AE2A2C
:10320000BF2A1D86E3C124E030E0A22AB32ADEC132
:103210004FE3C42E3E8531503E8783E68A8B44C1FE
:10322000F201C080FE85F150FE8722E030E0420EC0
:10323000531E3AC1F201C080D180892B49F0FD852F
:103240006F2F772767FD7095C6010E942C1B19C050
:10325000F60101900020E9F73197EC19E98B12C0D3
:10326000F201C080D180892B49F0FD856F2F77272F
:1032700067FD7095C6010E94211B03C0C6010E9414
:10328000181B898B22E030E0420E531E3E8589894F
:10329000381B3E8709C1A2FE08C0F20180819181DE
:1032A000A281B38124E030E009C0F20180819181E4
:1032B000AA2797FDA095BA2F22E030E0420E531EB8
:1032C0006C017D01B7FF0CC082E090E0A82AB92A0A
:1032D000F094E094D094C094C11CD11CE11CF11C6A
:1032E000EFEBFFEFAE22BF2221C020E430E0A22AA4
:1032F000B32A38E73A8B80E1898BA2FE08C0F2013D
:1033000080819181A281B38124E030E007C0F20185
:1033100080819181AA27BB2722E030E0420E531E14
:103320006C017D018FEC9FEFA822B9228701760105
:10333000FE013196F88BEF87F9896F2E7724882468
:103340009924C801B701A40193010E949B1B6A3014
:1033500024F02A89620F615201C0605DEF85F8890F
:103360006193F88BEF87C801B701A40193010E9414
:103370009B1B79018A01211531054105510509F78A
:10338000CC24DD247601CE010196CF84C81AC50174
:1033900082739070892B19F0FE85F150FE87A6FE8E
:1033A00009C02989203111F482E001C081E03E8505
:1033B000381B3E8738E0832E912C8A209B20A3FE69
:1033C0001BC08D85282F332727FD30958C2D9927FD
:1033D0008217930754F0E7EFFFEFAE22BF2228E0F9
:1033E000822E912C8A209B2007C0FD85FC19FD8729
:1033F0002E852F1B2E8703C03E853C193E87C501B5
:1034000080789170892B69F48E8506C0B10180E2C5
:1034100090E00E94371B812F182F11501816B4F31B
:103420001E87A1FE04C0B1018DE290E00BC0A4FE96
:1034300004C0B1018BE290E005C0A5FE05C0B1015A
:1034400080E290E00E94371BA6FE10C0B10180E32D
:1034500090E00E94371B8989803141F4B101EA89EB
:103460008E2F992787FD90950E94371BB0FE0DC0C7
:103470008E8506C0B10180E390E00E94371B812F4A
:10348000182F11501816B4F31E87892869F02D855E
:1034900006C0B10180E390E00E94371B212F122F5C
:1034A00011501216B4F31D8790E8692E712C6A2012
:1034B0007B20A7FC0DC08E8506C0B10180E290E0A4
:1034C0000E94371B812F182F11501816B4F31E8736
:1034D000FA89F33641F4B1018C2D992787FD909537
:1034E0000E94371B45C02A892337B1F44601560193
:1034F000198909C0F50181915F01B101992787FD03
:1035000090950E94371B1150A8F76401F989CF0EDE
:10351000D11C2FEF298B2CC03A89333519F00F8538
:1035200018891FC046018601B98808C0F801849136
:10353000B10199270E94371B0F5F1F4FBA94FFEF0D
:10354000BF16A1F764012989C20ED11CF98B10C0E6
:10355000F80182918F01B101992787FD90950E9412
:10356000371BCE0101960817190791F7188B0F87A3
:103570006728B1F08E8506C0B10180E290E00E941C
:10358000371B812F182F11501816B4F31E8708C04F
:10359000B101FA898F2F992787FD90950E94371BDB
:1035A000AA24BB2413C02A89253241F43AE0398B7E
:1035B0001E861D8681E0A82EB12C08C0B101EA89C3
:1035C0008E2F992787FD90950E94371B2B893C8968
:1035D0002F5F3F4F3C8B2B8BF101838183FF04C016
:1035E000EB89FC89F49103C0EB89FC89F081FA8BAB
:1035F0002A89222309F07ECDF10186819781649684
:103600000FB6F894DEBF0FBECDBFDF91CF911F91F3
:103610000F91FF90EF90DF90CF90BF90AF909F9071
:103620008F907F906F905F904F903F902F90089574
:10363000FC0105900020E9F7809590958E0F9F1F63
:103640000895FC010590615070400110D8F78095F5
:1036500090958E0F9F1F0895FC016150704001905E
:103660000110D8F7809590958E0F9F1F08950F93A6
:103670001F93CF93DF938C01EB018B81992781FFFF
:103680001BC082FF0DC02E813F818C819D81281738
:10369000390764F4E881F9810193F983E88306C06E
:1036A000E885F985802F0995892B31F48E819F81DA
:1036B00001969F838E8302C00FEF1FEFC801DF9139
:1036C000CF911F910F9108952F923F924F925F9249
:1036D0006F927F928F929F92AF92BF92CF92DF9222
:1036E000EF92FF920F931F93CF93DF93CDB7DEB787
:1036F000CA1BDB0B0FB6F894DEBF0FBECDBF09941B
:103700002A88398848885F846E847D848C849B8471
:10371000AA84B984C884DF80EE80FD800C811B817F
:10372000AA81B981CE0FD11D0FB6F894DEBF0FBEAE
:10373000CDBFED010895A1E21A2EAA1BBB1BFD010E
:103740000DC0AA1FBB1FEE1FFF1FA217B307E40780
:10375000F50720F0A21BB30BE40BF50B661F771FD8
:10376000881F991F1A9469F76095709580959095B8
:0C3770009B01AC01BD01CF010895FFCF0B
:10377C0041542B434D47523D4745545354415455A6
:10378C005347455452454C41593153455452454C7D
:10379C0041593147455452454C4159325345545285
:1037AC00454C41593247455454454D504E4F20439A
:1037BC004152524945524361206C205265616479F3
:1037CC00520049004E0047000D000000434D544983
:1037DC003A2022534D222C0041542B434D47533D4C
:1037EC00222B4F4B415445300041542B434D4746FF
:1037FC003D3100494E313D312C00494E313D302C8C
:10380C0000494E323D312C00494E323D302C005295
:10381C00454C4159313D312C0052454C4159313DBB
:10382C00302C0052454C4159323D312C0052454C04
:10383C004159323D302C0050494E41323D312C0023
:10384C0050494E41323D302C0050494E41313D31B2
:10385C002C0050494E41313D302C0050494E4130E6
:10386C003D312C0050494E41303D302C0050494EDA
:10387C0042373D312C0050494E42373D302C0050E0
:10388C00494E42363D312C0050494E42363D302C8B
:10389C000050494E42353D312C0050494E42353D89
:1038AC00302C0050494E42343D312C0050494E4290
:1038BC00343D302C0050494E42333D312C005049A0
:1038CC004E42333D302C0050494E42323D312C009B
:1038DC0050494E42323D302C0050494E42313D3120
:1038EC002C0050494E42313D302C0050494E423054
:1038FC003D312C0050494E42303D302C0042544E4C
:10390C003D312E0042544E3D302E000041542B438D
:10391C004D47523D256400436F6D6D616E642065AB
:10392C007865637574696F6E206661696C75726514
:0A393C000000000000000000000081
:00000001FF
